:10000000210AE2017E080A085D081F082B0837084C
:1000100067081A087F083B080E022D000602180E1A
:100020002E006E024D012F006F0610058F06300561
:100030000008000C2600180C06006100C30C02002A
:1000400000086F006D006E007000680069006A00B3
:100050006B006C00FA0C3100190911028101430791
:100060002D0AFA0CF101AA02190C8A0143072D0A84
:100070006A00AB020A0C8B014307540A6B00AC0206
:100080003C0C8C014307540A6C0009020801430729
:100090004B0A0000540A000028024307530A090CC7
:1000A0002800E900540AE8000C090B0243065B0A29
:1000B000050F43072D0A1007630A1004A8020A0C53
:1000C00088014306680030076B0A3004A9020A0C55
:1000D0008901430669000902010933000802010988
:1000E0003400090208014307770AA604780AA60526
:1000F0004306800A2B024307800AA605800C3401C0
:10010000100C3200740373030306880A0604890A7C
:10011000060500000000260500000000260400007F
:100120000000F202820A46050000460406042D0A79
:00000001FF
